:020000040800F2
:1000000000800020CD250008C5080008C7080008AA
:10001000C9080008CB080008CD080008000000004F
:10002000000000000000000000000000CF080008F1
:10003000D108000800000000D3080008D508000817
:100040001D2600081D2600081D2600081D26000884
:100050001D2600081D2600081D2600081D26000874
:100060001D2600081D2600081D2600081D26000864
:100070001D2600081D2600081D2600081D26000854
:100080001D2600081D2600081D2600081D26000844
:100090001D2600081D2600081D2600081D26000834
:1000A0001D2600081D2600081D2600081D26000824
:1000B0001D2600081D2600081D2600081D26000814
:1000C0001D2600081D2600081D2600081D26000804
:1000D0001D2600081D2600081D2600081D260008F4
:1000E0001D2600081D2600081D260008000000002F
:1000F0000000000000000000000000000000000000
:100100000000000000000000000000001D260008A4
:100110001D2600081D2600081D26000800000000FE
:100120001D2600081D2600081D2600081D260008A3
:100130001D26000800000000000000000000000074
:100140001D2600081D260008000000000000000019
:10015000000000000000000000000000000000009F
:1001600000000000000000001D2600081D260008F9
:100170001D26000800000000000000000000000034
:08018000000000001D2600082C
:1001880010B5054C237833B9044B13B10448AFF3C9
:1001980000800123237010BD0C0000200000000027
:1001A8007826000808B5034B1BB103490348AFF391
:1001B800008008BD0000000010000020782600081C
:1001C800F0B58BB00024059406940794089409941C
:1001D800364B5A6942F400225A615A6902F40022E5
:1001E8000192019A5A6942F480025A615A6902F4EA
:1001F80080020292029A5A6942F400325A615A699C
:1002080002F400320392039A5A6942F480225A6136
:100218005B6903F480230493049B224603214FF077
:10022800904000F09FFD224D22464FF42051284671
:1002380000F098FD4FF46043059303260696079453
:1002480005A91C4800F0AAFC059601270697079403
:10025800089405A94FF0904000F0A0FC44F2070371
:1002680005930694079405A9284600F097FC41F2E7
:10027800305305930696079405A9284600F08EFC8E
:100288004FF42053059306970794089405A9284628
:1002980000F084FC4FF4E06305930694079405A9E5
:1002A8004FF0904000F07AFC0BB0F0BD0010024017
:1002B800000400480008004872B6FEE708B50B487D
:1002C8000B4B03601023436000238360C36003610A
:1002D8004361037643768376C3760377437700F0EA
:1002E8004DFB00B908BDFFF7E7FF00BF0002002083
:1002F8000064004008B51148114B0360114B43607E
:10030800002383600122C260036143618361C3618A
:10031800036200F02CFD50B90021084800F085FD6B
:1003280038B90021054800F0AEFD20B908BDFFF737
:10033800C3FFFFF7C1FFFFF7BFFF00BFAC010020FD
:10034800005400400E09002008B50E480E4B03600B
:100358004FF482734360002383604FF44072C2609D
:10036800036143618361C36103624362836207225D
:10037800C26203630823436301F022FB00B908BD8E
:10038800FFF79AFF480100200030014010B596B0F1
:1003980000241394149415940C940D940E940F94B3
:1003A8001094119412942C22214601A802F033F9DA
:1003B8002548264B0360446084604FF6FF73C36092
:1003C80004614461846101F0D7FC002831D1002325
:1003D8001393159313A91C4801F0DAFD00282AD1BC
:1003E80060230C9300220D920E920F92109211929C
:1003F80012920CA9144801F02DFDF0B904220CA9A1
:10040800114801F027FDD0B900230193029303930B
:10041800049305934FF40052069207930B9301A996
:10042800094801F0F5FD60B9074800F0CDF916B0AC
:1004380010BDFFF741FFFFF73FFFFFF73DFFFFF755
:100448003BFFFFF739FF00BFB0000020004001402C
:1004580008B50B480B4B03604FF416434360002369
:100468008360C36003610C2242618361C3610362DC
:10047800436202F076F800B908BDFFF71DFF00BF20
:10048800280000200038014010B596B000241394CD
:10049800149415940C940D940E940F941094119434
:1004A80012942C22214601A802F0B5F82448254BC5
:1004B8000360446084604FF6FF73C3600461446165
:1004C800846101F059FC002832D10023139314935E
:1004D800159313A91A4801F05BFD00282AD160235F
:1004E8000C9300230D930E930F9310931193129373
:1004F80008220CA9124801F0ADFCE8B900230193C9
:1005080002930393049305934FF4005206920793C2
:1005180008934FF0007209920A930B9301A90848B7
:1005280001F076FD50B9064800F04EF916B010BD3E
:10053800FFF7C2FEFFF7C0FEFFF7BEFEFFF7BCFEE7
:10054800FC000020002C014000B59DB028220021AD
:1005580012A802F060F800210D910E910F911091F0
:1005680011913422684602F056F8022312930123AF
:1005780016931023179312A800F0B2FCC0B90F23EA
:100588000D9300210E910F91109111910DA800F07B
:10059800F7FF78B941F221030093002302930793F0
:1005A8000B93684601F0F2F830B91DB05DF804FB12
:1005B800FFF782FEFFF780FEFFF77EFE08B500F02A
:1005C800B9F9FFF7C1FFFFF7FBFDFFF777FEFFF76C
:1005D80091FEFFF7B9FEFFF7D9FEFFF739FFFFF7E6
:1005E80053FFFEE782B00A4B9A6942F001029A6112
:1005F8009A6902F001020092009ADA6942F0805288
:10060800DA61DB6903F080530193019B02B0704704
:100618000010024000B589B00023039304930593AA
:10062800069307930268144B9A4202D009B05DF80A
:1006380004FB03F5D633DA6942F00072DA61DA694D
:1006480002F000720192019A5A6942F400325A612A
:100658005B6903F400330293029B4FF4C053039386
:1006680002230493032306930923079303A94FF056
:10067800904000F093FAD9E700640040F0B589B0E3
:1006880000230393049305930693079302681E4B74
:100698009A4201D009B0F0BD1C4C636943F40033A1
:1006A8006361636903F400330093009B636943F457
:1006B80080236361636903F480230193019B4FF4F2
:1006C80000430393122704970326069604250795EB
:1006D80003A94FF0904000F061FA4FF400730393C0
:1006E8000497002305930696079503A9084800F088
:1006F80055FAE36943F40013E361E36903F4001373
:100708000293029BC6E700BF00540040001002405D
:100718000004004800B589B00023039304930593AF
:10072800069307930268144B9A4202D009B05DF809
:1007380004FB03F560439A6942F480529A619A690E
:1007480002F480520192019A5A6942F400325A61C5
:100758005B6903F400330293029BF02303930223A3
:100768000493032306930523079303A94FF09040AE
:1007780000F014FADAE700BF0030014082B00368E5
:100788000E4A934204D00E4A93420CD002B07047EE
:100798000C4B9A6942F400629A619B6903F4006306
:1007A8000093009BF2E7074B9A6942F480329A6102
:1007B8009B6903F480330193019BE7E7002C014018
:1007C800004001400010024000B589B000230393A7
:1007D800049305930693079303681A4A934205D036
:1007E800194A934218D009B05DF804FB174B5A69AF
:1007F80042F480225A615B6903F480230193019BD0
:100808004FF400430393022304930423079303A99B
:100818000F4800F0C3F9E6E70C4B5A6942F400327E
:100828005A615B6903F400330293029B0C23039320
:10083800022304930923079303A94FF0904000F083
:10084800ADF9D0E7002C0140004001400010024003
:100858000004004800B589B000230393049305936E
:10086800069307930268134B9A4202D009B05DF8C9
:1008780004FB03F558439A6942F480429A619A69E5
:1008880002F480420192019A5A6942F480225A6124
:100898005B6903F480230293029BC0230393022322
:1008A8000493032306930723079303A9024800F040
:1008B80075F9DBE70038014000040048FEE7FEE771
:1008C800FEE7FEE7FEE770477047704708B500F09F
:1008D80043F808BD034AD2F8883043F47003C2F8DD
:1008E8008830704700ED00E010B504460E4B1A78CA
:1008F8004FF47A73B3FBF2F30C4A1068B0FBF3F0D1
:1009080000F038F968B90F2C01D901200AE000225B
:1009180021464FF0FF3000F01DF9054B1C60002008
:1009280000E0012010BD00BF0400002000000020EE
:100938000800002008B5074A136843F01003136045
:10094800032000F0F5F80F20FFF7CEFFFFF74AFE6F
:10095800002008BD00200240034A1168034B1B78A1
:100968000B441360704700BF2802002004000020D9
:10097800014B1868704700BF28020020002800F0CB
:10098800A18038B5044690F82030D3B122681368A6
:1009980043F001031360FFF7EBFF054623685A682D
:1009A80012F0010F10D1FFF7E3FF401B0A28F5D919
:1009B800636A43F400336362052384F8203001201E
:1009C80038BDFFF727FEE1E71A6822F002021A6035
:1009D800FFF7CEFF054623685A6812F0020F0DD0C4
:1009E800FFF7C6FF401B0A28F5D9636A43F40033B2
:1009F8006362052384F820300120E1E7227E012A82
:100A08003DD01A6822F080021A60637E012B3BD029
:100A18002268136823F040031360A37E012B39D0AA
:100A28002268136823F020031360E37E012B37D07C
:100A38002268136843F010031360237F012B35D01D
:100A48002268136823F008031360637F012B33D0F7
:100A58002268136823F004031360A368E268134351
:100A680022691343626913436268013A2168134398
:100A7800CB6100206062012384F82030A0E71A6867
:100A880042F080021A60C0E72268136843F040030E
:100A98001360C2E72268136843F020031360C4E7B9
:100AA8002268136823F010031360C6E722681368EE
:100AB80043F008031360C8E72268136843F004038F
:100AC8001360CAE701207047002808DB0901C9B292
:100AD80000F1604000F5614080F80013704700F0B5
:100AE8000F000901C9B2014B1954704714ED00E019
:100AF80000B500F00700C0F1070CBCF1040F28BFD7
:100B08004FF0040C031D062B0FD9C31E4FF0FF3EF8
:100B18000EFA0CF021EA000199400EFA03FE22EACF
:100B28000E0241EA02005DF804FB0023EEE7000034
:100B3800074AD36823F4E0631B041B0C000200F48B
:100B4800E060034343F0BF6343F40033D36070476E
:100B580000ED00E010B50446054BD868C0F302204C
:100B6800FFF7C6FF01462046FFF7AEFF10BD00BFE6
:100B780000ED00E00138B0F1807F0BD24FF0E023A8
:100B88005861054AF02182F8231000209861072255
:100B98001A6170470120704700ED00E0F0B583B09E
:100BA800002362E085685E000324B44025EA04055A
:100BB800CC68B4402C438460456825EA0C054C6831
:100BC800C4F300149C402C4344605FE0DD08083502
:100BD80050F8254003F0070C4FEA8C0C4FF00F0E2D
:100BE8000EFA0CFE24EA0E0E0C6904FA0CF444EA20
:100BF8000E0440F8254060E0042400E0002404FAD4
:100C08000EF42C430CF1020C524D45F82C40524C7A
:100C1800A568D44325EA02064F6817F4801F01D05F
:100C280042EA05064C4DAE60ED6804EA05064F68D9
:100C380017F4001F01D042EA0506474DEE606D68C3
:100C480004EA05064F6817F4003F01D042EA05069A
:100C5800414D6E602D682C404E6816F4803F01D0DF
:100C680042EA05043C4A146001330A6832FA03F484
:100C78006ED04FF0010C0CFA03FC1CEA0202F3D010
:100C88004C6804F00304013C012C8BD94C6804F037
:100C98000304032C0CD0C4685D004FF0030C0CFA5D
:100CA80005FC24EA0C0C8C68AC4044EA0C04C460D3
:100CB8004C6804F00304022C88D004684FEA430E01
:100CC8004FF0030C0CFA0EFC24EA0C0C4C6804F0F0
:100CD800030404FA0EF444EA0C0404604C6814F4A7
:100CE800403FC1D01D4CA56945F00105A561A46927
:100CF80004F001040194019C4FEA930C0CF10205E5
:100D0800144C54F8255003F0030E4FEA8E0E0F24AE
:100D180004FA0EF425EA0405B0F1904F3FF46EAFE3
:100D28000F4CA0420ED004F58064A0420CD004F50C
:100D38008064A0420AD004F58064A0423FF45CAF0E
:100D480005245CE701245AE7022458E7032456E700
:100D580003B0F0BD00000140000401400010024053
:100D6800000400480AB18161704781627047002819
:100D780059D010B5044690F84130002B43D02423B5
:100D880084F841302268136823F001031360636814
:100D9800226823F0706313612268936823F4004388
:100DA8009360E368012B33D0A368226843F40443BB
:100DB8009360E368022B31D02268536843F00073D4
:100DC80043F4004353602268D36823F40043D3609C
:100DD800236962691343A169226843EA0123D36046
:100DE800E369216A22680B4313602268136843F0A1
:100DF8000103136000206064202384F841302063DD
:100E080084F8420010BD80F84030FFF737FCB6E7A1
:100E1800A368226843F400439360CAE723684FF449
:100E280000625A60C8E701207047034690F84120E5
:100E3800D2B2202A23D190F84020012A21D00122C1
:100E480080F84020242280F841200068026822F0BF
:100E5800010202601868026822F480520260186871
:100E680002681143016019680A6842F001020A60C9
:100E7800202283F84120002083F840007047022098
:100E8800704702207047034690F84120D2B2202ACA
:100E980021D190F84020012A1FD0012280F840205B
:100EA800242280F841200068026822F001020260D2
:100EB8001868026822F4706242EA01220260196826
:100EC8000A6842F001020A60202283F841200020CB
:100ED80083F84000704702207047022070470000E6
:100EE800002800F0FF8270B582B00446036813F052
:100EF800010F3BD0B44B5B6803F00C03042B1ED0EE
:100F0800B14B5B6803F00C03082B13D06368B3F58F
:100F1800803F68D0002B40F0928003F1804303F5B6
:100F280004331A6822F480321A601A6822F4802284
:100F38001A605DE0A44B5B6813F4803FE6D04FF481
:100F4800003393FAA3F3A04B19684FF4003393FAD4
:100F5800A3F3B3FA83F303F01F03012202FA03F3A6
:100F68000B4203D06368002B00F0BE82236813F0A5
:100F7800020F00F0C480944B5B6813F00C0F00F074
:100F88009C80914B5B6803F00C03082B00F08F806A
:100F98002369002B00F0F080012292FAA2F3B3FA41
:100FA80083F303F1845303F584139B001A60FFF75E
:100FB800DFFC0546022393FAA3F3834B1968022347
:100FC80093FAA3F3B3FA83F303F01F03012202FA9F
:100FD80003F30B4240F0C280FFF7CAFC401B022813
:100FE800E8D9032089E2784A136843F48033136010
:100FF800754AD36A23F00F03A1680B43D362636871
:10100800002B36D0FFF7B4FC05464FF4003393FAB3
:10101800A3F36D4B19684FF4003393FAA3F3B3FAB3
:1010280083F303F01F03012202FA03F30B429DD15D
:10103800FFF79EFC401B6428E7D903205DE2B3F567
:10104800A02F09D0604B1A6822F480321A601A68FF
:1010580022F480221A60CBE703F18043A3F53C33E6
:101068001A6842F480221A601A6842F480321A60C0
:10107800BEE7FFF77DFC05464FF4003393FAA3F370
:10108800514B19684FF4003393FAA3F3B3FA83F37F
:1010980003F01F03012202FA03F30B423FF466AF89
:1010A800FFF766FC401B6428E6D9032025E2464B7F
:1010B8005B6813F4803F7FF46BAF022393FAA3F3CA
:1010C800414B1968022393FAA3F3B3FA83F303F0AD
:1010D8001F03012202FA03F30B4203D02369934250
:1010E80040F004823848036823F0F8036169F82265
:1010F80092FAA2F2B2FA82F291400B43036023689B
:1011080013F0080F00F08C80A369002B60D0012138
:1011180091FAA1F2B2FA82F22C4B13449B001960A7
:10112800FFF726FC0546022393FAA3F293FAA3F2EB
:1011380093FAA3F2244A516A93FAA3F3B3FA83F316
:1011480003F01F03012202FA03F30B4268D1FFF7F1
:101158000FFC401B0228E6D90320CEE11A48036899
:1011680023F0F8036169F82292FAA2F2B2FA82F245
:1011780091400B430360C2E7012393FAA3F3B3FA48
:1011880083F303F1845303F584139B0000221A6050
:10119800FFF7EEFB0546022393FAA3F30A4B1968FF
:1011A800022393FAA3F3B3FA83F303F01F03012294
:1011B80002FA03F30B42A2D0FFF7DAFB401B022826
:1011C800E9D9032099E100BF001002402081901066
:1011D800012292FAA2F2B2FA82F2B74B13449B00B0
:1011E80000221A60FFF7C4FB0546022393FAA3F214
:1011F80093FAA3F293FAA3F2B04A516A93FAA3F3CB
:10120800B3FA83F303F01F03012202FA03F30B423C
:1012180006D0FFF7ADFB401B0228E6D903206CE19E
:10122800236813F0040F00F0A980A44BDB6913F0C6
:10123800805F20D1A14BDA6942F08052DA61DB6924
:1012480003F080530193019B01259D4B1B6813F408
:10125800807F12D0E368012B23D073BB03F1804356
:1012680003F504331A6A22F001021A621A6A22F09C
:1012780004021A621AE00025E7E7914A136843F46A
:1012880080731360FFF774FB06468D4B1B6813F4DD
:10129800807FDFD1FFF76CFB801B6428F5D9032022
:1012A8002BE1864A136A43F001031362E368002BBB
:1012B8003CD0FFF75DFB06462EE0052B09D07F4B9F
:1012C8001A6A22F001021A621A6A22F004021A62E9
:1012D800ECE77A4B1A6A42F004021A621A6A42F080
:1012E80001021A62E2E7022393FAA3F3734B596AE5
:1012F800022393FAA3F3B3FA83F303F01F03012243
:1013080002FA03F3194238D1FFF732FB801B41F28E
:101318008833984200F2EC80022393FAA3F293FAFE
:10132800A3F3002BDFD0654B196AE1E7FFF720FB39
:10133800064618E0022393FAA3F3604B596A022386
:1013480093FAA3F3B3FA83F303F01F03012202FA1B
:1013580003F3194211D0FFF70BFB801B41F28833CE
:10136800984200F2C780022393FAA3F293FAA3F3F8
:10137800002BDFD0514B196AE1E7B5BBE369002BBD
:1013880000F0BA804D4A526802F00C02082A00F0B8
:101398009980022B2FD04FF0807393FAA3F3B3FAFE
:1013A80083F303F1845303F584139B0000221A602E
:1013B800FFF7DEFA04464FF0007393FAA3F33F4BAE
:1013C80019684FF0007393FAA3F3B3FA83F303F0A9
:1013D8001F03012202FA03F319426BD0FFF7C8FA80
:1013E800001B0228E7D9032087E0344AD36923F099
:1013F8008053D361C2E74FF0807393FAA3F3B3FA33
:1014080083F303F1845303F584139B0000221A60CD
:10141800FFF7AEFA05464FF0007393FAA3F3274B94
:1014280019684FF0007393FAA3F3B3FA83F303F048
:101438001F03012202FA03F3194206D0FFF798FAB4
:10144800401B0228E7D9032057E01C494B6823F4C6
:101458007413626A206A024313434B604FF080732F
:1014680093FAA3F3B3FA83F303F1845303F58413D4
:101478009B0001221A60FFF77BFA04464FF00073C5
:1014880093FAA3F30D4B19684FF0007393FAA3F383
:10149800B3FA83F303F01F03012202FA03F319429C
:1014A80006D1FFF765FA001B0228E7D9032024E0DC
:1014B800002022E0002020E020819010001002404F
:1014C80000700040012B1AD0104B5B6803F4803188
:1014D800226A914215D103F47013626A934212D1C1
:1014E80000200AE001207047012006E0012004E006
:1014F800032002E0032000E0002002B070BD0120BC
:10150800FBE70120F9E70120F7E700BF00100240E0
:10151800164B5B6803F00C02082A01D01448704788
:1015280003F470114FF4701292FAA2F2B2FA82F236
:1015380021FA02F20F49885C0C4AD26A02F00F02C3
:101548000F2191FAA1F1B1FA81F1CA400A498A5CE6
:1015580013F4803F05D0064BB3FBF2F303FB00F016
:101568007047064B03FB00F0704700BF00100240B5
:1015780000127A00B8260008A826000800093D00D5
:10158800002800F0BE8070B50D460446614B1B680C
:1015980003F007038B420BD25E4A136823F007035C
:1015A8000B431360136803F007038B4240F0AB80D2
:1015B800236813F0020F06D0574A536823F0F0034C
:1015C800A1680B435360236813F0010F5AD0636876
:1015D800012B2DD0022B40D0022292FAA2F24E4AC1
:1015E8001068022292FAA2F2B2FA82F202F01F0204
:1015F800012101FA02F2104200F0878046494A6848
:1016080022F0030213434B60FFF7B2F90646424B40
:101618005B6803F00C036268B3EB820F32D0FFF70C
:10162800A7F9801B41F288339842F0D9032067E07C
:101638004FF4003292FAA2F2374A10684FF400329F
:1016480092FAA2F2B2FA82F202F01F02012101FA22
:1016580002F20242D2D1012052E04FF0007292FA17
:10166800A2F22D4A10684FF0007292FAA2F2B2FA72
:1016780082F202F01F02012101FA02F21042BDD1EA
:1016880001203DE0234B1B6803F00703AB420AD956
:10169800204A136823F007032B431360136803F0F1
:1016A8000703AB4233D1236813F0040F06D01A4A5C
:1016B800536823F4E063E1680B435360236813F035
:1016C800080F07D0144A536823F46053216943EA8A
:1016D800C1035360FFF71CFF0F4B5B6803F0F00377
:1016E800F02292FAA2F2B2FA82F2D3400B4AD35C09
:1016F800D8400B4B18600B4B1868FFF7F5F8002023
:1017080070BD012070470120FAE70120F8E70120A9
:10171800F6E700BF002002400010024098260008AB
:101728000000002008000020014B1868704700BF27
:101738000000002008B5FFF7F7FF074B5B6803F4CC
:10174800E0634FF4E06292FAA2F2B2FA82F2D34076
:10175800024AD35CD84008BD001002409026000819
:1017680008B5FFF7E1FF074B5B6803F460534FF4DC
:10177800605292FAA2F2B2FA82F2D340024AD35CE1
:10178800D84008BD0010024090260008F0B583B08C
:101798000446036813F4803F48D0864BDB6913F096
:1017A800805F40F0BE80834BDA6942F08052DA6194
:1017B800DB6903F080530193019B01257E4B1B6875
:1017C80013F4807F00F0AF807A4B1B6A13F44073E8
:1017D80022D0626802F440729A421DD07548016AAC
:1017E80021F440764FF4803393FAA3F2B2FA82F2EE
:1017F800724F3A4492004FF0010CC2F800C093FABD
:10180800A3F3B3FA83F33B449B0000221A600662F9
:1018180011F0010F40F09C80664A136A23F440736C
:1018280061680B431362002D40F0B980236813F000
:10183800010F06D05F4A136B23F00303A1680B4323
:101848001363236813F0020F06D05A4A136B23F46C
:101858004033E1680B431363236813F0040F06D089
:10186800544A136B23F4402321690B431363236801
:1018780013F0200F06D04F4A136B23F01003E169D1
:101888000B431363236813F4003F06D0494A536897
:1018980023F48003216B0B435360236813F0400F3C
:1018A80006D0444A136B23F02003216A0B431363C9
:1018B800236813F0080F06D03E4A136B23F4401335
:1018C80061690B431363236813F0100F06D0394A7C
:1018D800136B23F44003A1690B431363236813F4C8
:1018E800007F06D0334A536823F40003A16A0B43F0
:1018F8005360236813F0800F06D02E4AD36A23F46E
:10190800F873616A0B43D362236813F4805F4DD088
:10191800284A136B23F48073E16A0B431363002096
:1019280045E000254AE7244A136843F480731360AE
:10193800FFF71EF80646204B1B6813F4807F7FF4E0
:1019480043AFFFF715F8801B6428F4D903202EE075
:10195800FFF70EF8064618E0022393FAA3F3154B97
:10196800596A022393FAA3F3B3FA83F303F01F032C
:10197800012202FA03F30B427FF44EAFFEF7F8FFA1
:10198800801B41F2883398420ED8022393FAA3F2BF
:1019980093FAA3F3002BDFD0064B196AE1E7D3696A
:1019A80023F08053D36141E7032000E0002003B017
:1019B800F0BD00BF00100240007000400081901090
:1019C80000286FD010B50446436A33B94368B3F5AD
:1019D800827F05D00023C36102E0002303614361D5
:1019E8000023A36294F85D30002B52D0022384F8C0
:1019F8005D302268136823F040031360E368B3F591
:101A0800E06F4CD90022B3F5706F04D0B3F5E06FE6
:101A180001D00023A362636803F48273A16801F410
:101A280004410B43216901F002010B43616901F094
:101A380001010B43A16901F400710B43E16901F055
:101A480038010B43216A01F080010B43A16A01F4BC
:101A5800005120680B430360638B03F00403616A41
:101A680001F010010B43616B01F008010B43E168C1
:101A780001F470610B43216813434B602268D369FA
:101A880023F40063D36100202066012384F85D30CD
:101A980010BD84F85C302046FEF73CFEA6E74FF404
:101AA8008052B0E70120704730B4036A23F0010385
:101AB8000362026A4468836923F4803323F0730362
:101AC8000D681D4322F002028B681343184A9042A6
:101AD8000BD002F5A052904207D002F580629042E6
:101AE80003D002F58062904205D123F00803CA684A
:101AF8001A4322F004030E4A90420BD002F5A0527A
:101B0800904207D002F58062904203D002F58062CD
:101B1800904205D124F440744A6922438C691443E5
:101B2800446085614A684263036230BC704700BF05
:101B3800002C014030B4036A23F480730362036A03
:101B48004268C46924F4803C2CF0730C0C6844EAA5
:101B58000C0523F400738C6843EA0423124CA0425A
:101B68000BD0124CA0420FD004F58064A0420BD0D9
:101B780004F58064A0420FD106E023F40063CC682A
:101B880043EA042323F4806322F440524C6942EA76
:101B980004128C6942EA04124260C5614A68C26351
:101BA800036230BC704700BF002C01400040014078
:101BB80030B4036A23F480530362026A4468C36939
:101BC80023F0807323F4E6430D6843EA052322F4E7
:101BD80000528D6842EA05320D4DA8420BD005F53A
:101BE800A055A84207D005F58065A84203D005F5A1
:101BF8008065A84204D124F480444D6944EA8514E0
:101C08004460C3614B680364026230BC704700BF24
:101C1800002C014030B4036A23F480330362036A62
:101C28004468426D22F4803222F070020D682A4323
:101C380023F400338D6843EA05430D4DA8420BD0C9
:101C480005F5A055A84207D005F58065A84203D040
:101C580005F58065A84204D124F480344D6944EA2E
:101C68000524446042654A688265036230BC704757
:101C7800002C014030B4036A23F480130362026A23
:101C88004468436D23F0807323F4E0430D6843EA0E
:101C9800052322F400128D6842EA05520D4DA84230
:101CA8000BD005F5A055A84207D005F58065A842D8
:101CB80003D005F58065A84204D124F480244D6939
:101CC80044EA8524446043654B68C365026230BCBE
:101CD800704700BF002C01400368264A90420AD092
:101CE800B0F1804F07D0A2F59432904203D002F5AC
:101CF8008062904203D123F070034A6813431D4A5F
:101D0800904216D0B0F1804F13D0A2F59432904291
:101D18000FD002F5806290420BD002F59C329042BF
:101D280007D002F58062904203D002F580629042AB
:101D380003D123F44073CA68134323F080034A692C
:101D4800134303608B68C3620B688362094B984234
:101D58000BD003F5A053984207D003F5806398424F
:101D680003D003F58063984201D10B690363012313
:101D780043617047002C014060B310B5044690F8E9
:101D88003D3013B3022384F83D30214651F8040B4B
:101D9800FFF7A2FF012384F8483084F83E3084F826
:101DA8003F3084F8403084F8413084F8423084F879
:101DB800433084F8443084F8453084F8463084F859
:101DC800473084F83D30002010BD80F83C30FEF7E5
:101DD800D5FCD7E70120704730B4036A23F010031D
:101DE8000362036A4268846924F0807C2CF4E64C20
:101DF8000C684CEA042423F020038D6843EA051399
:101E0800124DA8420BD0124DA8420FD005F580659F
:101E1800A8420BD005F58065A8420FD106E023F053
:101E28008003CD6843EA051323F0400322F440629F
:101E38004D6942EA85028D6942EA85024260846101
:101E48004A688263036230BC704700BF002C0140BF
:101E58000040014038B590F83C30012B00F09580E7
:101E680004460D46012380F83C30142A00F288808D
:101E7800DFE802F00B8686861F868686348686868D
:101E8800488686865D86868671000068FFF70CFEA8
:101E98002268936943F0080393612268936923F0E9
:101EA800040393612268936929690B4393610020B5
:101EB80067E00068FFF790FF2268936943F40063C6
:101EC80093612268936923F480639361226893691C
:101ED800296943EA01239361002052E00068FFF773
:101EE80029FE2268D36943F00803D3612268D369C5
:101EF80023F00403D3612268D36929690B43D361B2
:101F080000203EE00068FFF753FE2268D36943F4DF
:101F18000063D3612268D36923F48063D3612268A4
:101F2800D369296943EA0123D361002029E00068C5
:101F3800FFF770FE2268536D43F00803536522686B
:101F4800536D23F0040353652268536D29690B43CD
:101F58005365002015E00068FFF78CFE2268536D7A
:101F680043F4006353652268536D23F4806353651B
:101F78002268536D296943EA01235365002000E074
:101F88000120002384F83C3038BD0220FCE7000023
:101F980090F83C20012A37D030B40346012280F85B
:101FA8003C20022280F83D20006842688468174D72
:101FB800A84224D022F070020D682A4342601A68B1
:101FC800124882420ED0B2F1804F0BD0A0F5943067
:101FD800824207D000F58060824203D000F59C3031
:101FE800824204D124F0800489682143916001224F
:101FF80083F83D20002083F83C0030BC704722F471
:1020080070024D682A43D5E702207047002C014032
:1020180090F83C30012B3BD010B40246012380F8E5
:102028003C30CB6823F440738868034323F480630F
:102038004868034323F400630868034323F4805388
:102048000869034323F400534869034323F4804396
:10205800886A034323F47023886943EA00431068BD
:102068000C4CA04206D04364002082F83C005DF886
:10207800044B704723F470034C6A43EA045323F07B
:102088008073CC69234323F00073096A0B43EAE7A2
:1020980002207047002C0140026852E8003F23F4F8
:1020A800907342E800310029F6D1026802F1080372
:1020B80053E8003F23F00103083242E800310029C9
:1020C800F3D1036E012B06D02023C0F88030002303
:1020D800036683667047026852E8003F23F01003E6
:1020E80042E800310029F6D1EEE7000010B50446B9
:1020F800836802691A4343691A43C3691A4301682A
:102108000B6823F4164323F00C0313430B60026897
:10211800536823F44053C1680B4353608269036AD0
:102128001A4301688B6823F4306313438B60036898
:102138007B4A93421BD07B4A93422AD07A4A9342E5
:102148003BD07A4A93424BD0794A93425BD01023D2
:10215800E069B0F5004F00F08B80082B00F2DA80C0
:10216800DFE803F0B3C9B1D8CCD8D8D8CF00714BC9
:102178001B6B03F00303032B09D8DFE803F0020409
:1021880006570123E4E70423E2E70823E0E71023E6
:10219800DEE7684B1B6B03F44033B3F5003F47D0D1
:1021A80006D8002B46D0B3F5803F45D10423CFE7AE
:1021B800B3F5403F42D10223CAE75E4B1B6B03F4E1
:1021C8004023B3F5002F3BD005D8DBB3B3F5802F00
:1021D8003AD10423BCE7B3F5402F37D10223B7E740
:1021E800544B1B6B03F44013B3F5001F30D005D8D4
:1021F80083B3B3F5801F2FD10423A9E7B3F5401F9C
:102208002CD10223A4E74B4B1B6B03F44003B3F51B
:10221800000F25D005D82BB3B3F5800F24D10423A4
:1022280096E7B3F5400F21D1022391E702238FE708
:1022380008238DE700238BE7102389E7102387E71E
:10224800082385E7002383E7102381E710237FE72E
:1022580008237DE700237BE7102379E7102377E73E
:10226800082375E7002373E7102371E710236FE74E
:10227800082B49D8DFE803F0051F254822484848BD
:102288000900FFF757FA002840D06268530803EBAB
:102298004003B3FBF2F3A3F110014FF6EF72914242
:1022A80036D89AB222F00F02C3F3420313432268CE
:1022B800D36000201BE0FFF753FAE4E7FFF728F9A3
:1022C800E1E71D48E1E71C4802E0FFF733FA18B3DD
:1022D800636800EB5300B0FBF3F0A0F110024FF677
:1022E800EF739A421AD8236880B2D860002000237E
:1022F800A366E36610BDFFF733FAE8E7FFF708F9CE
:10230800E5E74FF40040E3E70120F0E70020EEE7BF
:102318000120ECE70120EAE70020E8E70120E6E7F2
:10232800003801400044004000480040004C004094
:10233800005000400010024000127A00436A13F077
:10234800010F06D00268536823F40033816A0B43F7
:102358005360436A13F0020F06D00268536823F4EF
:102368008033C16A0B435360436A13F0040F06D0ED
:102378000268536823F48023016B0B435360436A5C
:1023880013F0080F06D00268536823F40043416B2A
:102398000B435360436A13F0100F06D0026893682A
:1023A80023F48053816B0B439360436A13F0200F2F
:1023B80006D00268936823F40053C16B0B43936003
:1023C800436A13F0400F0AD00268536823F480135D
:1023D800016C0B435360036CB3F5801F0BD0436A49
:1023E80013F0800F06D00268536823F40023816C31
:1023F8000B43536070470268536823F4C003416C71
:102408000B435360EBE72DE9F84305460F461646A4
:102418009946DDF820802B68DC6937EA04040CBF94
:1024280001240024B44232D1B8F1FF3FF3D0FEF7C3
:102438009FFAA0EB090040452CD8B8F1000F2BD02B
:102448002B681A6812F0040FE5D0DA6912F0080F49
:1024580011D1DA6912F4006FDDD04FF400621A620C
:102468002846FFF719FE2023C5F88430002385F895
:10247800783003200CE008241C622846FFF70CFE85
:10248800C5F88440002385F87830012000E000205A
:10249800BDE8F8830320FBE70320F9E730B583B0F4
:1024A80004460023C0F88430FEF762FA0546226825
:1024B800126812F0080F0FD123681B6813F0040F7D
:1024C80026D12023E367C4F88030002020666066A8
:1024D80084F8780003B030BD6FF07E430093034664
:1024E80000224FF400112046FFF78DFF0028E3D0AB
:1024F800226852E8003F23F0800342E800310029B7
:10250800F6D12023E367002384F878300320E1E73D
:102518006FF07E4300932B4600224FF48001204643
:10252800FFF771FF0028CCD0226852E8003F23F45F
:10253800907342E800310029F6D1226802F10803BD
:1025480053E8003F23F00103083242E80031002934
:10255800F3D12023C4F88030002384F87830032096
:10256800B8E768B310B50446C36F03B32423E36721
:102578002268136823F0010313602046FFF7B6FDB5
:10258800012813D0636ABBB92268536823F49043C7
:1025980053602268936823F02A03936022681368C3
:1025A80043F0010313602046FFF778FF10BD80F861
:1025B8007830FEF74FF9D9E72046FFF7BFFEE3E78B
:1025C80001207047DFF834D0FEF784F90C480D4934
:1025D8000D4A002302E0D458C4500433C4188C4276
:1025E800F9D30A4A0A4C002301E013600432A242DC
:1025F800FBD300F019F8FDF7E1FFFEE700800020AB
:10260800000000200C000020D02600080C0000204C
:102618002C020020FEE702440346934200D1704793
:1026280003F8011BF9E7000070B50D4D0D4C641B54
:10263800A4100026A64209D10B4D0C4C00F018F846
:10264800641BA4100026A64205D170BD55F8043BB2
:1026580098470136EEE755F8043B98470136F2E70C
:10266800C8260008C8260008C8260008CC26000886
:10267800F8B500BFF8BC08BC9E467047F8B500BF67
:08268800F8BC08BC9E46704737
:102690000000000001020304000000000000000030
:1026A00001020304060708090102030405060708DE
:1026B000090A0B0C0D0E0F1002030405060708098A
:0826C0000A0B0C0D0E0F1010A7
:0426C800AD01000858
:0426CC008901000878
:0C26D00000127A00010000001000000061
:04000005080025CDFD
:00000001FF
